:020000040000FA
:100000002500DE0C0200080C0600000C26004B0C3C
:100010002D006607090A6A00AA02FB0966060C0A97
:10002000ED02090A6B006C00010C27000A0229008E
:1000300030002800080C2E00310A6607290A070242
:100040004307260AA7026800A8024F0AA802000078
:100050004F0A070243064C0A670008022900080CF1
:100060002E000902F00103043003100229000A02E5
:1000700089002D000306430A6D02AD02080C8D00B5
:100080000306720A940A010C8D000307B30A080CD8
:100090008D000306DC0ABE0A0000000000000C020E
:1000A000E20100007F0A9F0A0000B30A000000007E
:1000B0000000000000000000000000000000000040
:1000C0000000C90A0000000000000000000000005D
:1000D0000000000000000000000000000000000020
:1000E0000000E90A080CAD00010C2C000D020F0EF7
:1000F000A3050009A3042B002F00AF027F0A000014
:1001000000000000EE028B0A080C2E000B022F00EC
:10011000AF0200001D0AEF02910AAF02020C260096
:100120001D0A0C0226001D0A020C2C000D020F0EE7
:10013000A3050009A3042B002F00AF02A10A0000B1
:100140000000EE02AA0A080C2E000B022F00AF02DC
:1001500000001D0AEF02B00AAF02040C26001D0ABF
:100160000C0226001D0A040C2C00040C26000000C2
:10017000000000000000000000001D0A100C2C0010
:100180000D020F0EA3050009A3042B002F00AF02E0
:10019000CA0A0000EE02D30A080C2E000B022F0040
:1001A000AF0200001D0AEF02D90AAF02040C2600BC
:1001B0001D0A0C0226001D0A080CAD00200C2C00A4
:1001C0000D020F0EA3050009A3042B002F00AF02A0
:1001D000E90AEE02F20A080C2E000B022F00AF0211
:1001E00000001D0AEF02F80AAF02100C26001D0ADB
:1001F0000C0226001D0A050C3100F102FD0A000068
:06020000000000000008F0
:10040000E2010008010802080308040805080608BC
:10041000070808080808080808080808080808085D
:020420000808CA
:021FFE00EA0FE8
:00000001FF
